******************************************************************************
             TMS320C2000 Linker PC v16.9.4                     
******************************************************************************
>> Linked Wed Jan 03 13:19:46 2018

OUTPUT FILE NAME:   <SourceCode_C28.out>
ENTRY POINT SYMBOL: "_c_int00"  address: 0013f46d


MEMORY CONFIGURATION

         name            origin    length      used     unused   attr    fill
----------------------  --------  ---------  --------  --------  ----  --------
PAGE 0:
  RAML0                 00008000   00001000  0000006a  00000f96  RWIX
  RAML1                 00009000   00001000  00000000  00001000  RWIX
  FLASHG                00120000   00008000  00000000  00008000  RWIX
  FLASHF                00128000   00008000  00000000  00008000  RWIX
  FLASHE                00130000   00008000  00000000  00008000  RWIX
  FLASHD                00138000   00002000  0000006a  00001f96  RWIX
  FLASHC                0013a000   00002000  00000000  00002000  RWIX
  FLASHA                0013e000   00001f80  00001f55  0000002b  RWIX
  CSM_RSVD              0013ff80   00000070  00000000  00000070  RWIX
  BEGIN                 0013fff0   00000002  00000002  00000000  RWIX
  FLASH_EXE_ONLY_P0     0013fff2   00000002  00000000  00000002  RWIX
  ECSL_PWL_P0           0013fff4   00000004  00000000  00000004  RWIX
  CSM_PWL_P0            0013fff8   00000008  00000000  00000008  RWIX
  FPUTABLES             003fd258   000006a0  00000000  000006a0  RWIX
  IQTABLES              003fd8f8   00000b50  00000000  00000b50  RWIX
  IQTABLES2             003fe448   0000008c  00000000  0000008c  RWIX
  IQTABLES3             003fe4d4   000000aa  00000000  000000aa  RWIX
  BOOTROM               003feda8   00001200  00000000  00001200  RWIX
  PIEMISHNDLR           003fffbe   00000002  00000000  00000002  RWIX
  RESET                 003fffc0   00000002  00000000  00000002  RWIX
  VECTORS               003fffc2   0000003e  00000000  0000003e  RWIX

PAGE 1:
  BOOT_RSVD             00000002   000001a0  00000000  000001a0  RWIX
  RAMM0                 000001a2   0000025e  00000000  0000025e  RWIX
  RAMM1                 00000400   00000400  00000300  00000100  RWIX
  DEV_EMU               00000880   00000180  00000042  0000013e  RWIX
  CSM                   00000ae0   00000020  00000016  0000000a  RWIX
  ADC1_RESULT           00000b00   00000020  00000010  00000010  RWIX
  ADC2_RESULT           00000b40   00000020  00000010  00000010  RWIX
  CPU_TIMER0            00000c00   00000008  00000008  00000000  RWIX
  CPU_TIMER1            00000c08   00000008  00000008  00000000  RWIX
  CPU_TIMER2            00000c10   00000008  00000008  00000000  RWIX
  PIE_CTRL              00000ce0   00000020  0000001a  00000006  RWIX
  PIE_VECT              00000d00   00000100  00000100  00000000  RWIX
  PIE_VECT_CP           00000e00   00000100  00000100  00000000  RWIX
  DMA                   00001000   00000200  000000e0  00000120  RWIX
  ASYSCTRLCONFIG        00001700   00000080  00000078  00000008  RWIX
  FLASH_REGS            00004000   00000300  00000182  0000017e  RWIX
  FLASH_ECC             00004300   00000040  00000024  0000001c  RWIX
  M3PLL                 00004400   00000010  00000008  00000008  RWIX
  EPI_REGS              00004430   00000010  0000000c  00000004  RWIX
  RAM_REGS              00004900   00000080  0000003e  00000042  RWIX
  RAM_ERR_REGS          00004a00   00000080  0000003e  00000042  RWIX
  CM_MC_IPC             00004e00   00000040  00000040  00000000  RWIX
  MCBSPA                00005000   00000040  00000024  0000001c  RWIX
  EPWM1                 00005100   00000080  00000080  00000000  RWIX
  EPWM2                 00005180   00000080  00000080  00000000  RWIX
  EPWM3                 00005200   00000080  00000080  00000000  RWIX
  EPWM4                 00005280   00000080  00000080  00000000  RWIX
  EPWM5                 00005300   00000080  00000080  00000000  RWIX
  EPWM6                 00005380   00000080  00000080  00000000  RWIX
  EPWM7                 00005400   00000080  00000080  00000000  RWIX
  EPWM8                 00005480   00000080  00000080  00000000  RWIX
  EPWM9                 00005500   00000080  00000080  00000000  RWIX
  ECAP1                 00005a00   00000020  00000020  00000000  RWIX
  ECAP2                 00005a20   00000020  00000020  00000000  RWIX
  ECAP3                 00005a40   00000020  00000020  00000000  RWIX
  ECAP4                 00005a60   00000020  00000020  00000000  RWIX
  ECAP5                 00005a80   00000020  00000020  00000000  RWIX
  ECAP6                 00005aa0   00000020  00000020  00000000  RWIX
  EQEP1                 00005b00   00000040  00000022  0000001e  RWIX
  EQEP2                 00005b40   00000040  00000022  0000001e  RWIX
  EQEP3                 00005b80   00000040  00000022  0000001e  RWIX
  GPIOG1CTRL            00005f80   00000040  00000040  00000000  RWIX
  GPIOG1DAT             00005fc0   00000020  00000020  00000000  RWIX
  GPIOG1TRIP            00005fe0   00000020  00000020  00000000  RWIX
  COMP1                 00006400   00000020  00000007  00000019  RWIX
  COMP2                 00006420   00000020  00000007  00000019  RWIX
  COMP3                 00006440   00000020  00000007  00000019  RWIX
  COMP4                 00006460   00000020  00000007  00000019  RWIX
  COMP5                 00006480   00000020  00000007  00000019  RWIX
  COMP6                 000064a0   00000020  00000007  00000019  RWIX
  GPIOG2CTRL            00006f80   00000040  0000003c  00000004  RWIX
  GPIOG2DAT             00006fc0   00000020  00000020  00000000  RWIX
  SYSTEM                00007010   00000020  0000001d  00000003  RWIX
  SPIA                  00007040   00000010  00000010  00000000  RWIX
  SCIA                  00007050   00000010  00000010  00000000  RWIX
  NMIINTRUPT            00007060   00000010  00000006  0000000a  RWIX
  XINTRUPT              00007070   00000010  00000010  00000000  RWIX
  ADC1                  00007100   00000080  00000050  00000030  RWIX
  ADC2                  00007180   00000080  00000050  00000030  RWIX
  I2CA                  00007900   00000040  00000022  0000001e  RWIX
  RAML2                 0000a000   00001000  000005f2  00000a0e  RWIX
  RAML3                 0000b000   00001000  00000000  00001000  RWIX
  RAMS0                 0000c000   00001000  00000000  00001000  RWIX
  RAMS1                 0000d000   00001000  00000000  00001000  RWIX
  RAMS2                 0000e000   00001000  00000000  00001000  RWIX
  RAMS3                 0000f000   00001000  00000000  00001000  RWIX
  RAMS4                 00010000   00001000  00000000  00001000  RWIX
  RAMS5                 00011000   00001000  00000000  00001000  RWIX
  RAMS6                 00012000   00001000  00000000  00001000  RWIX
  RAMS7                 00013000   00001000  00000000  00001000  RWIX
  CTOMRAM               0003f800   00000380  00000088  000002f8  RWIX
  MTOCRAM               0003fc00   00000380  00000000  00000380  RWIX
  FLASHB                0013c000   00002000  00000000  00002000  RWIX
  FLASH_EXE_ONLY        0013fff2   00000002  00000002  00000000  RWIX
  ECSL_PWL              0013fff4   00000004  00000004  00000000  RWIX
  CSM_PWL               0013fff8   00000008  00000008  00000000  RWIX


SECTION ALLOCATION MAP

 output                                  attributes/
section   page    origin      length       input sections
--------  ----  ----------  ----------   ----------------
.TI.ramfunc 
*          0    00138000    0000006a     RUN ADDR = 00008000
                  00138000    00000066     F28M35x_SysCtrl.obj (.TI.ramfunc)
                  00138066    00000004     F28M35x_usDelay.obj (.TI.ramfunc)

.text      0    0013e000    00001611     
                  0013e000    0000048c     F28M35x_Init.obj (.text)
                  0013e48c    000003bc     F28M35x_Ipc.obj (.text)
                  0013e848    0000035f     F28M35x_DefaultIsr.obj (.text:retain)
                  0013eba7    000002bb     SCI_Debug.obj (.text)
                  0013ee62    00000194     main.obj (.text:retain)
                  0013eff6    0000011a     F28M35x_SysCtrl.obj (.text)
                  0013f110    000000e4     Concerto_C2x_IPC.obj (.text:retain)
                  0013f1f4    000000d2     adc.obj (.text:retain)
                  0013f2c6    00000099     F28M35x_Ipc_Util.obj (.text)
                  0013f35f    00000093     Concerto_C2x_IPC.obj (.text)
                  0013f3f2    0000007b     F28M35x_CpuTimers.obj (.text)
                  0013f46d    00000056     rts2800_fpu32.lib : boot28.obj (.text)
                  0013f4c3    00000043     main.obj (.text)
                  0013f506    0000002d     F28M35x_PieCtrl.obj (.text)
                  0013f533    00000029     rts2800_fpu32.lib : exit.obj (.text)
                  0013f55c    00000024     F28M35x_Gpio.obj (.text)
                  0013f580    00000024     rts2800_fpu32.lib : cpy_tbl.obj (.text)
                  0013f5a4    00000020     F28M35x_PieVect.obj (.text)
                  0013f5c4    0000001e     rts2800_fpu32.lib : memcpy.obj (.text)
                  0013f5e2    00000019                       : args_main.obj (.text)
                  0013f5fb    0000000a                       : strcmp.obj (.text)
                  0013f605    00000009                       : _lock.obj (.text)
                  0013f60e    00000002                       : pre_init.obj (.text)
                  0013f610    00000001                       : startup.obj (.text)

.econst    0    0013f614    00000630     
                  0013f614    00000258     SCI_Debug.obj (.econst:_$P$T4$5)
                  0013f86c    00000226     SCI_Debug.obj (.econst:_$P$T1$2)
                  0013fa92    00000100     F28M35x_PieVect.obj (.econst:_PieVectTableInit)
                  0013fb92    00000041     SCI_Debug.obj (.econst:.string)
                  0013fbd3    0000002a     SCI_Debug.obj (.econst:.string:_$P$T0$1)
                  0013fbfd    0000002a     SCI_Debug.obj (.econst:.string:_$P$T2$3)
                  0013fc27    0000001d     SCI_Debug.obj (.econst:.string:_$P$T3$4)

.cinit     0    0013fc44    00000314     
                  0013fc44    000002c3     SCI_Debug.obj (.cinit)
                  0013ff07    0000002a     main.obj (.cinit)
                  0013ff31    0000000e     rts2800_fpu32.lib : exit.obj (.cinit)
                  0013ff3f    0000000d     Concerto_C2x_IPC.obj (.cinit)
                  0013ff4c    00000005     rts2800_fpu32.lib : _lock.obj (.cinit:__lock)
                  0013ff51    00000005                       : _lock.obj (.cinit:__unlock)
                  0013ff56    00000002     --HOLE-- [fill = 0]

codestart 
*          0    0013fff0    00000002     
                  0013fff0    00000002     F28M35x_CodeStartBranch.obj (codestart)

.stack     1    00000400    00000300     UNINITIALIZED
                  00000400    00000300     --HOLE--

DevEmuRegsFile 
*          1    00000880    00000042     UNINITIALIZED
                  00000880    00000042     F28M35x_GlobalVariableDefs.obj (DevEmuRegsFile)

CsmRegsFile 
*          1    00000ae0    00000016     UNINITIALIZED
                  00000ae0    00000016     F28M35x_GlobalVariableDefs.obj (CsmRegsFile)

AdcResultFile 
*          1    00000b00    00000010     UNINITIALIZED
                  00000b00    00000010     F28M35x_GlobalVariableDefs.obj (AdcResultFile)

Adc1ResultFile 
*          1    00000b00    00000010     UNINITIALIZED
                  00000b00    00000010     F28M35x_GlobalVariableDefs.obj (Adc1ResultFile)

Adc2ResultFile 
*          1    00000b40    00000010     UNINITIALIZED
                  00000b40    00000010     F28M35x_GlobalVariableDefs.obj (Adc2ResultFile)

CpuTimer0RegsFile 
*          1    00000c00    00000008     UNINITIALIZED
                  00000c00    00000008     F28M35x_GlobalVariableDefs.obj (CpuTimer0RegsFile)

CpuTimer1RegsFile 
*          1    00000c08    00000008     UNINITIALIZED
                  00000c08    00000008     F28M35x_GlobalVariableDefs.obj (CpuTimer1RegsFile)

CpuTimer2RegsFile 
*          1    00000c10    00000008     UNINITIALIZED
                  00000c10    00000008     F28M35x_GlobalVariableDefs.obj (CpuTimer2RegsFile)

PieCtrlRegsFile 
*          1    00000ce0    0000001a     UNINITIALIZED
                  00000ce0    0000001a     F28M35x_GlobalVariableDefs.obj (PieCtrlRegsFile)

PieVectTableFile 
*          1    00000d00    00000100     UNINITIALIZED
                  00000d00    00000100     F28M35x_GlobalVariableDefs.obj (PieVectTableFile)

EmuKeyVar 
*          1    00000d00    00000000     UNINITIALIZED

EmuBModeVar 
*          1    00000d00    00000000     UNINITIALIZED

FlashCallbackVar 
*          1    00000d00    00000000     UNINITIALIZED

FlashScalingVar 
*          1    00000d00    00000000     UNINITIALIZED

PieVectTableCopyFile 
*          1    00000e00    00000100     UNINITIALIZED
                  00000e00    00000100     F28M35x_GlobalVariableDefs.obj (PieVectTableCopyFile)

DmaRegsFile 
*          1    00001000    000000e0     UNINITIALIZED
                  00001000    000000e0     F28M35x_GlobalVariableDefs.obj (DmaRegsFile)

AnalogSysctrlRegsFile 
*          1    00001700    00000078     UNINITIALIZED
                  00001700    00000078     F28M35x_GlobalVariableDefs.obj (AnalogSysctrlRegsFile)

FlashCtrlRegsFile 
*          1    00004000    00000182     UNINITIALIZED
                  00004000    00000182     F28M35x_GlobalVariableDefs.obj (FlashCtrlRegsFile)

FlashEccRegsFile 
*          1    00004300    00000024     UNINITIALIZED
                  00004300    00000024     F28M35x_GlobalVariableDefs.obj (FlashEccRegsFile)

M3PllRegsFile 
*          1    00004400    00000008     UNINITIALIZED
                  00004400    00000008     F28M35x_GlobalVariableDefs.obj (M3PllRegsFile)

EpiRegsFile 
*          1    00004430    0000000c     UNINITIALIZED
                  00004430    0000000c     F28M35x_GlobalVariableDefs.obj (EpiRegsFile)

RAMRegsFile 
*          1    00004900    0000003e     UNINITIALIZED
                  00004900    0000003e     F28M35x_GlobalVariableDefs.obj (RAMRegsFile)

RAMErrRegsFile 
*          1    00004a00    0000003e     UNINITIALIZED
                  00004a00    0000003e     F28M35x_GlobalVariableDefs.obj (RAMErrRegsFile)

CtoMIpcRegsFile 
*          1    00004e00    00000040     UNINITIALIZED
                  00004e00    00000040     F28M35x_GlobalVariableDefs.obj (CtoMIpcRegsFile)

McbspaRegsFile 
*          1    00005000    00000024     UNINITIALIZED
                  00005000    00000024     F28M35x_GlobalVariableDefs.obj (McbspaRegsFile)

EPwm1RegsFile 
*          1    00005100    00000080     UNINITIALIZED
                  00005100    00000080     F28M35x_GlobalVariableDefs.obj (EPwm1RegsFile)

EPwm2RegsFile 
*          1    00005180    00000080     UNINITIALIZED
                  00005180    00000080     F28M35x_GlobalVariableDefs.obj (EPwm2RegsFile)

EPwm3RegsFile 
*          1    00005200    00000080     UNINITIALIZED
                  00005200    00000080     F28M35x_GlobalVariableDefs.obj (EPwm3RegsFile)

EPwm4RegsFile 
*          1    00005280    00000080     UNINITIALIZED
                  00005280    00000080     F28M35x_GlobalVariableDefs.obj (EPwm4RegsFile)

EPwm5RegsFile 
*          1    00005300    00000080     UNINITIALIZED
                  00005300    00000080     F28M35x_GlobalVariableDefs.obj (EPwm5RegsFile)

EPwm6RegsFile 
*          1    00005380    00000080     UNINITIALIZED
                  00005380    00000080     F28M35x_GlobalVariableDefs.obj (EPwm6RegsFile)

EPwm7RegsFile 
*          1    00005400    00000080     UNINITIALIZED
                  00005400    00000080     F28M35x_GlobalVariableDefs.obj (EPwm7RegsFile)

EPwm8RegsFile 
*          1    00005480    00000080     UNINITIALIZED
                  00005480    00000080     F28M35x_GlobalVariableDefs.obj (EPwm8RegsFile)

EPwm9RegsFile 
*          1    00005500    00000080     UNINITIALIZED
                  00005500    00000080     F28M35x_GlobalVariableDefs.obj (EPwm9RegsFile)

ECap1RegsFile 
*          1    00005a00    00000020     UNINITIALIZED
                  00005a00    00000020     F28M35x_GlobalVariableDefs.obj (ECap1RegsFile)

ECap2RegsFile 
*          1    00005a20    00000020     UNINITIALIZED
                  00005a20    00000020     F28M35x_GlobalVariableDefs.obj (ECap2RegsFile)

ECap3RegsFile 
*          1    00005a40    00000020     UNINITIALIZED
                  00005a40    00000020     F28M35x_GlobalVariableDefs.obj (ECap3RegsFile)

ECap4RegsFile 
*          1    00005a60    00000020     UNINITIALIZED
                  00005a60    00000020     F28M35x_GlobalVariableDefs.obj (ECap4RegsFile)

ECap5RegsFile 
*          1    00005a80    00000020     UNINITIALIZED
                  00005a80    00000020     F28M35x_GlobalVariableDefs.obj (ECap5RegsFile)

ECap6RegsFile 
*          1    00005aa0    00000020     UNINITIALIZED
                  00005aa0    00000020     F28M35x_GlobalVariableDefs.obj (ECap6RegsFile)

EQep1RegsFile 
*          1    00005b00    00000022     UNINITIALIZED
                  00005b00    00000022     F28M35x_GlobalVariableDefs.obj (EQep1RegsFile)

EQep2RegsFile 
*          1    00005b40    00000022     UNINITIALIZED
                  00005b40    00000022     F28M35x_GlobalVariableDefs.obj (EQep2RegsFile)

EQep3RegsFile 
*          1    00005b80    00000022     UNINITIALIZED
                  00005b80    00000022     F28M35x_GlobalVariableDefs.obj (EQep3RegsFile)

GpioCtrlRegsFile 
*          1    00005f80    00000040     UNINITIALIZED
                  00005f80    00000040     F28M35x_GlobalVariableDefs.obj (GpioCtrlRegsFile)

GpioG1CtrlRegsFile 
*          1    00005f80    00000040     UNINITIALIZED
                  00005f80    00000040     F28M35x_GlobalVariableDefs.obj (GpioG1CtrlRegsFile)

GpioDataRegsFile 
*          1    00005fc0    00000020     UNINITIALIZED
                  00005fc0    00000020     F28M35x_GlobalVariableDefs.obj (GpioDataRegsFile)

GpioG1DataRegsFile 
*          1    00005fc0    00000020     UNINITIALIZED
                  00005fc0    00000020     F28M35x_GlobalVariableDefs.obj (GpioG1DataRegsFile)

GpioTripRegsFile 
*          1    00005fe0    00000020     UNINITIALIZED
                  00005fe0    00000020     F28M35x_GlobalVariableDefs.obj (GpioTripRegsFile)

GpioG1TripRegsFile 
*          1    00005fe0    00000020     UNINITIALIZED
                  00005fe0    00000020     F28M35x_GlobalVariableDefs.obj (GpioG1TripRegsFile)

Comp1RegsFile 
*          1    00006400    00000007     UNINITIALIZED
                  00006400    00000007     F28M35x_GlobalVariableDefs.obj (Comp1RegsFile)

Comp2RegsFile 
*          1    00006420    00000007     UNINITIALIZED
                  00006420    00000007     F28M35x_GlobalVariableDefs.obj (Comp2RegsFile)

Comp3RegsFile 
*          1    00006440    00000007     UNINITIALIZED
                  00006440    00000007     F28M35x_GlobalVariableDefs.obj (Comp3RegsFile)

Comp4RegsFile 
*          1    00006460    00000007     UNINITIALIZED
                  00006460    00000007     F28M35x_GlobalVariableDefs.obj (Comp4RegsFile)

Comp5RegsFile 
*          1    00006480    00000007     UNINITIALIZED
                  00006480    00000007     F28M35x_GlobalVariableDefs.obj (Comp5RegsFile)

Comp6RegsFile 
*          1    000064a0    00000007     UNINITIALIZED
                  000064a0    00000007     F28M35x_GlobalVariableDefs.obj (Comp6RegsFile)

GpioG2CtrlRegsFile 
*          1    00006f80    0000003c     UNINITIALIZED
                  00006f80    0000003c     F28M35x_GlobalVariableDefs.obj (GpioG2CtrlRegsFile)

GpioG2DataRegsFile 
*          1    00006fc0    00000020     UNINITIALIZED
                  00006fc0    00000020     F28M35x_GlobalVariableDefs.obj (GpioG2DataRegsFile)

SysCtrlRegsFile 
*          1    00007010    0000001d     UNINITIALIZED
                  00007010    0000001d     F28M35x_GlobalVariableDefs.obj (SysCtrlRegsFile)

SpiaRegsFile 
*          1    00007040    00000010     UNINITIALIZED
                  00007040    00000010     F28M35x_GlobalVariableDefs.obj (SpiaRegsFile)

SciaRegsFile 
*          1    00007050    00000010     UNINITIALIZED
                  00007050    00000010     F28M35x_GlobalVariableDefs.obj (SciaRegsFile)

NmiIntruptRegsFile 
*          1    00007060    00000006     UNINITIALIZED
                  00007060    00000006     F28M35x_GlobalVariableDefs.obj (NmiIntruptRegsFile)

XIntruptRegsFile 
*          1    00007070    00000010     UNINITIALIZED
                  00007070    00000010     F28M35x_GlobalVariableDefs.obj (XIntruptRegsFile)

AdcRegsFile 
*          1    00007100    00000050     UNINITIALIZED
                  00007100    00000050     F28M35x_GlobalVariableDefs.obj (AdcRegsFile)

Adc1RegsFile 
*          1    00007100    00000050     UNINITIALIZED
                  00007100    00000050     F28M35x_GlobalVariableDefs.obj (Adc1RegsFile)

Adc2RegsFile 
*          1    00007180    00000050     UNINITIALIZED
                  00007180    00000050     F28M35x_GlobalVariableDefs.obj (Adc2RegsFile)

I2caRegsFile 
*          1    00007900    00000022     UNINITIALIZED
                  00007900    00000022     F28M35x_GlobalVariableDefs.obj (I2caRegsFile)

FlashExeOnlyFile 
*          1    0013fff2    00000002     UNINITIALIZED
                  0013fff2    00000002     F28M35x_GlobalVariableDefs.obj (FlashExeOnlyFile)

EcslPwlFile 
*          1    0013fff4    00000004     UNINITIALIZED
                  0013fff4    00000004     F28M35x_GlobalVariableDefs.obj (EcslPwlFile)

CsmPwlFile 
*          1    0013fff8    00000008     UNINITIALIZED
                  0013fff8    00000008     F28M35x_GlobalVariableDefs.obj (CsmPwlFile)

.pinit     0    0013e000    00000000     UNINITIALIZED

PUTBUFFER 
*          1    0003f800    00000080     UNINITIALIZED
                  0003f800    00000080     F28M35x_Ipc.obj (PUTBUFFER)

PUTWRITEIDX 
*          1    0003f880    00000004     UNINITIALIZED
                  0003f880    00000004     F28M35x_Ipc.obj (PUTWRITEIDX)

GETREADIDX 
*          1    0003f884    00000004     UNINITIALIZED
                  0003f884    00000004     F28M35x_Ipc.obj (GETREADIDX)

GETBUFFER 
*          0    0003fc00    00000080     DSECT
                  0003fc00    00000080     F28M35x_Ipc.obj (GETBUFFER)

GETWRITEIDX 
*          0    0003fc80    00000004     DSECT
                  0003fc80    00000004     F28M35x_Ipc.obj (GETWRITEIDX)

PUTREADIDX 
*          0    0003fc84    00000004     DSECT
                  0003fc84    00000004     F28M35x_Ipc.obj (PUTREADIDX)

.ebss      1    0000a000    000005f2     UNINITIALIZED
                  0000a000    0000038b     SCI_Debug.obj (.ebss)
                  0000a38b    00000001     --HOLE--
                  0000a38c    00000018     F28M35x_CpuTimers.obj (.ebss)
                  0000a3a4    00000006     rts2800_fpu32.lib : exit.obj (.ebss)
                  0000a3aa    00000002     F28M35x_Init.obj (.ebss)
                  0000a3ac    00000002     rts2800_fpu32.lib : _lock.obj (.ebss:__lock)
                  0000a3ae    00000002                       : _lock.obj (.ebss:__unlock)
                  0000a3b0    00000010     --HOLE--
                  0000a3c0    000000d4     adc.obj (.ebss)
                  0000a494    0000002c     --HOLE--
                  0000a4c0    000000a4     Concerto_C2x_IPC.obj (.ebss)
                  0000a564    0000001c     --HOLE--
                  0000a580    00000072     main.obj (.ebss)

.reset     0    003fffc0    00000002     DSECT
                  003fffc0    00000002     rts2800_fpu32.lib : boot28.obj (.reset)

vectors    0    003fffc2    00000000     DSECT

MODULE SUMMARY

       Module                           code   initialized data   uninitialized data
       ------                           ----   ----------------   ------------------
    .\
       SCI_Debug.obj                    699    2035               907               
       F28M35x_Init.obj                 1164   0                  2                 
       F28M35x_Ipc.obj                  956    0                  136               
       F28M35x_DefaultIsr.obj           863    0                  0                 
       main.obj                         471    42                 114               
       Concerto_C2x_IPC.obj             375    13                 164               
       F28M35x_SysCtrl.obj              486    0                  0                 
       adc.obj                          210    0                  212               
       F28M35x_PieVect.obj              32     256                0                 
       F28M35x_Ipc_Util.obj             153    0                  0                 
       F28M35x_CpuTimers.obj            123    0                  24                
       F28M35x_PieCtrl.obj              45     0                  0                 
       F28M35x_Gpio.obj                 36     0                  0                 
       F28M35x_usDelay.obj              8      0                  0                 
       F28M35x_CodeStartBranch.obj      2      0                  0                 
    +--+--------------------------------+------+------------------+--------------------+
       Total:                           5623   2346               1559              
                                                                                    
    .\source\
       F28M35x_GlobalVariableDefs.obj   0      0                  3915              
    +--+--------------------------------+------+------------------+--------------------+
       Total:                           0      0                  3915              
                                                                                    
    C:\ti\ccsv7\tools\compiler\ti-cgt-c2000_16.9.4.LTS\lib\rts2800_fpu32.lib
       boot28.obj                       86     0                  0                 
       exit.obj                         41     14                 6                 
       cpy_tbl.obj                      36     0                  0                 
       memcpy.obj                       30     0                  0                 
       args_main.obj                    25     0                  0                 
       _lock.obj                        9      10                 4                 
       strcmp.obj                       10     0                  0                 
       pre_init.obj                     2      0                  0                 
       startup.obj                      1      0                  0                 
    +--+--------------------------------+------+------------------+--------------------+
       Total:                           240    24                 10                
                                                                                    
       Stack:                           0      0                  768               
    +--+--------------------------------+------+------------------+--------------------+
       Grand Total:                     5863   2370               6252              


GLOBAL DATA SYMBOLS: SORTED BY DATA PAGE

address     data page           name
--------    ----------------    ----
00000400      10 (00000400)     __stack

00000880      22 (00000880)     _DevEmuRegs

00000ae0      2b (00000ac0)     _CsmRegs

00000b00      2c (00000b00)     _Adc1Result
00000b00      2c (00000b00)     _AdcResult

00000b40      2d (00000b40)     _Adc2Result

00000c00      30 (00000c00)     _CpuTimer0Regs
00000c08      30 (00000c00)     _CpuTimer1Regs
00000c10      30 (00000c00)     _CpuTimer2Regs

00000ce0      33 (00000cc0)     _PieCtrlRegs

00000d00      34 (00000d00)     _PieVectTable

00000e00      38 (00000e00)     _PieVectTableCopy

00001000      40 (00001000)     _DmaRegs

00001700      5c (00001700)     _AnalogSysctrlRegs

00004000     100 (00004000)     _FlashCtrlRegs

00004300     10c (00004300)     _FlashEccRegs

00004400     110 (00004400)     _M3PllRegs
00004430     110 (00004400)     _EpiRegs

00004900     124 (00004900)     _RAMRegs

00004a00     128 (00004a00)     _RAMErrRegs

00004e00     138 (00004e00)     _CtoMIpcRegs

00005000     140 (00005000)     _McbspaRegs

00005100     144 (00005100)     _EPwm1Regs

00005180     146 (00005180)     _EPwm2Regs

00005200     148 (00005200)     _EPwm3Regs

00005280     14a (00005280)     _EPwm4Regs

00005300     14c (00005300)     _EPwm5Regs

00005380     14e (00005380)     _EPwm6Regs

00005400     150 (00005400)     _EPwm7Regs

00005480     152 (00005480)     _EPwm8Regs

00005500     154 (00005500)     _EPwm9Regs

00005a00     168 (00005a00)     _ECap1Regs
00005a20     168 (00005a00)     _ECap2Regs

00005a40     169 (00005a40)     _ECap3Regs
00005a60     169 (00005a40)     _ECap4Regs

00005a80     16a (00005a80)     _ECap5Regs
00005aa0     16a (00005a80)     _ECap6Regs

00005b00     16c (00005b00)     _EQep1Regs

00005b40     16d (00005b40)     _EQep2Regs

00005b80     16e (00005b80)     _EQep3Regs

00005f80     17e (00005f80)     _GpioCtrlRegs
00005f80     17e (00005f80)     _GpioG1CtrlRegs

00005fc0     17f (00005fc0)     _GpioDataRegs
00005fc0     17f (00005fc0)     _GpioG1DataRegs
00005fe0     17f (00005fc0)     _GpioG1TripRegs
00005fe0     17f (00005fc0)     _GpioTripRegs

00006400     190 (00006400)     _Comp1Regs
00006420     190 (00006400)     _Comp2Regs

00006440     191 (00006440)     _Comp3Regs
00006460     191 (00006440)     _Comp4Regs

00006480     192 (00006480)     _Comp5Regs
000064a0     192 (00006480)     _Comp6Regs

00006f80     1be (00006f80)     _GpioG2CtrlRegs

00006fc0     1bf (00006fc0)     _GpioG2DataRegs

00007010     1c0 (00007000)     _SysCtrlRegs

00007040     1c1 (00007040)     _SpiaRegs
00007050     1c1 (00007040)     _SciaRegs
00007060     1c1 (00007040)     _NmiIntruptRegs
00007070     1c1 (00007040)     _XIntruptRegs

00007100     1c4 (00007100)     _Adc1Regs
00007100     1c4 (00007100)     _AdcRegs

00007180     1c6 (00007180)     _Adc2Regs

00007900     1e4 (00007900)     _I2caRegs

0000a000     280 (0000a000)     _enModuleTest
0000a001     280 (0000a000)     _MS_Delay
0000a002     280 (0000a000)     _aInitMsg
0000a017     280 (0000a000)     _aADC1TestSuccess

0000a040     281 (0000a040)     _aFailGPIOInputTest
0000a058     281 (0000a040)     _aADC1TestFail

0000a080     282 (0000a080)     _aADC1Test
0000a09a     282 (0000a080)     _aSuccessGPIOInputTest

0000a0c0     283 (0000a0c0)     _aStartGPIOInputTest

0000a100     284 (0000a100)     _aADC1ChannelTest

0000a140     285 (0000a140)     _aStartTestMsg

0000a180     286 (0000a180)     _aRxBufferSCI

0000a1c0     287 (0000a1c0)     _aEndTestMsg

0000a240     289 (0000a240)     _aStartMsg

0000a38c     28e (0000a380)     _CpuTimer1
0000a394     28e (0000a380)     _CpuTimer2
0000a39c     28e (0000a380)     _CpuTimer0
0000a3a4     28e (0000a380)     ___TI_enable_exit_profile_output
0000a3a6     28e (0000a380)     ___TI_cleanup_ptr
0000a3a8     28e (0000a380)     ___TI_dtors_ptr
0000a3aa     28e (0000a380)     _FAULT_WARNING
0000a3ac     28e (0000a380)     __lock
0000a3ae     28e (0000a380)     __unlock

0000a3c0     28f (0000a3c0)     _ConversionCount
0000a3c1     28f (0000a3c0)     _ConversionCount1
0000a3c2     28f (0000a3c0)     _adc2Voltage_ChannelA7
0000a3cc     28f (0000a3c0)     _adc1Voltage_ChannelA7
0000a3d6     28f (0000a3c0)     _adc2Voltage_ChannelB0
0000a3e0     28f (0000a3c0)     _adc1Voltage_ChannelA6
0000a3ea     28f (0000a3c0)     _adc2Voltage_ChannelA4
0000a3f4     28f (0000a3c0)     _adc1Voltage_ChannelB0

0000a400     290 (0000a400)     _adc2Voltage_ChannelB3
0000a40a     290 (0000a400)     _adc1Voltage_ChannelB7
0000a414     290 (0000a400)     _adc2Voltage_ChannelB4
0000a41e     290 (0000a400)     _adc1Voltage_ChannelB3
0000a428     290 (0000a400)     _adc2Voltage_ChannelA6
0000a432     290 (0000a400)     _adc1Voltage_ChannelB4

0000a440     291 (0000a440)     _adc1Voltage_ChannelA2
0000a44a     291 (0000a440)     _adc2Voltage_ChannelA2
0000a454     291 (0000a440)     _adc1Voltage_ChannelA0
0000a45e     291 (0000a440)     _adc2Voltage_ChannelA0
0000a468     291 (0000a440)     _adc1Voltage_ChannelA4
0000a472     291 (0000a440)     _adc2Voltage_ChannelB7

0000a480     292 (0000a480)     _adc1Voltage_ChannelA3
0000a48a     292 (0000a480)     _adc2Voltage_ChannelA3

0000a4c0     293 (0000a4c0)     _IPCDataReceiveFlag
0000a4c1     293 (0000a4c0)     _ErrorFlag
0000a4c2     293 (0000a4c0)     _pulMsgRam
0000a4c4     293 (0000a4c0)     _pulMsgRam_M3
0000a4c6     293 (0000a4c0)     _g_sIpcController1
0000a4d4     293 (0000a4c0)     _g_sIpcController2

0000a500     294 (0000a500)     _IPCRecievedBuffer

0000a580     296 (0000a580)     _ErrorCount
0000a581     296 (0000a580)     _tempVal
0000a582     296 (0000a580)     _timerOut
0000a583     296 (0000a580)     _loop
0000a584     296 (0000a580)     _LoopCount
0000a585     296 (0000a580)     _i
0000a586     296 (0000a580)     _count
0000a587     296 (0000a580)     _counter
0000a588     296 (0000a580)     _dataStore
0000a58a     296 (0000a580)     _dataStore1
0000a58c     296 (0000a580)     _ipcData

0000a5c0     297 (0000a5c0)     _rdata

0003f800     fe0 (0003f800)     _g_asIPCCtoMBuffers

0003f880     fe2 (0003f880)     _g_usPutWriteIndexes
0003f884     fe2 (0003f880)     _g_usGetReadIndexes

0003fc00     ff0 (0003fc00)     _g_asIPCMtoCBuffers

0003fc80     ff2 (0003fc80)     _g_usGetWriteIndexes
0003fc84     ff2 (0003fc80)     _g_usPutReadIndexes

0013fa92    4fea (0013fa80)     _PieVectTableInit

0013fff2    4fff (0013ffc0)     _FlashExeOnly
0013fff4    4fff (0013ffc0)     _EcslPwl
0013fff8    4fff (0013ffc0)     _CsmPwl


GLOBAL SYMBOLS: SORTED ALPHABETICALLY BY Name 

page  address   name                            
----  -------   ----                            
0     0013e000  .text                           
0     0013f533  C$$EXIT                         
0     0013e906  _ADCINT1_ISR                    
0     0013e910  _ADCINT2_ISR                    
0     0013eadc  _ADCINT3_ISR                    
0     0013eae6  _ADCINT4_ISR                    
0     0013eaf0  _ADCINT5_ISR                    
0     0013eafa  _ADCINT6_ISR                    
0     0013eb04  _ADCINT7_ISR                    
0     0013eb0e  _ADCINT8_ISR                    
0     0013ec15  _ADC_Test                       
0     0013f33c  _AckIpcFlag                     
0     0013e034  _Adc1Config                     
1     00007100  _Adc1Regs                       
1     00000b00  _Adc1Result                     
0     0013e0a8  _Adc2Config                     
1     00007180  _Adc2Regs                       
1     00000b40  _Adc2Result                     
1     00007100  _AdcRegs                        
1     00000b00  _AdcResult                      
0     0013e152  _AdcSocPWM                      
1     00001700  _AnalogSysctrlRegs              
0     0013eb54  _CFLFSM_ISR                     
0     0013eb4a  _CFLSINGERR_ISR                 
0     0013eb68  _CRAMACCVIOL_ISR                
0     0013eb5e  _CRAMSINGERR_ISR                
0     0013f0f8  _CSMSecurityStatus              
1     00006400  _Comp1Regs                      
1     00006420  _Comp2Regs                      
1     00006440  _Comp3Regs                      
1     00006460  _Comp4Regs                      
1     00006480  _Comp5Regs                      
1     000064a0  _Comp6Regs                      
0     0013f433  _ConfigCpuTimer                 
1     0000a3c0  _ConversionCount                
1     0000a3c1  _ConversionCount1               
1     0000a39c  _CpuTimer0                      
1     00000c00  _CpuTimer0Regs                  
1     0000a38c  _CpuTimer1                      
1     00000c08  _CpuTimer1Regs                  
1     0000a394  _CpuTimer2                      
1     00000c10  _CpuTimer2Regs                  
1     0013fff8  _CsmPwl                         
1     00000ae0  _CsmRegs                        
0     0013f0a5  _CsmUnlock                      
1     00004e00  _CtoMIpcRegs                    
0     0013e85c  _DATALOG_ISR                    
0     0013ea78  _DINTCH1_ISR                    
0     0013ea82  _DINTCH2_ISR                    
0     0013ea8c  _DINTCH3_ISR                    
0     0013ea96  _DINTCH4_ISR                    
0     0013eaa0  _DINTCH5_ISR                    
0     0013eaaa  _DINTCH6_ISR                    
0     00008066  _DSP28x_usDelay                 
1     00000880  _DevEmuRegs                     
1     00001000  _DmaRegs                        
0     0013e9e2  _ECAP1_INT_ISR                  
0     0013e9ec  _ECAP2_INT_ISR                  
0     0013e9f6  _ECAP3_INT_ISR                  
0     0013ea00  _ECAP4_INT_ISR                  
0     0013ea0a  _ECAP5_INT_ISR                  
0     0013ea14  _ECAP6_INT_ISR                  
0     0013f104  _ECSLSecurityStatus             
1     00005a00  _ECap1Regs                      
1     00005a20  _ECap2Regs                      
1     00005a40  _ECap3Regs                      
1     00005a60  _ECap4Regs                      
1     00005a80  _ECap5Regs                      
1     00005aa0  _ECap6Regs                      
0     0013eb86  _EMPTY_ISR                      
0     0013e870  _EMUINT_ISR                     
0     0013e992  _EPWM1_INT_ISR                  
0     0013e942  _EPWM1_TZINT_ISR                
0     0013e99c  _EPWM2_INT_ISR                  
0     0013e94c  _EPWM2_TZINT_ISR                
0     0013e9a6  _EPWM3_INT_ISR                  
0     0013e956  _EPWM3_TZINT_ISR                
0     0013e9b0  _EPWM4_INT_ISR                  
0     0013e960  _EPWM4_TZINT_ISR                
0     0013e9ba  _EPWM5_INT_ISR                  
0     0013e96a  _EPWM5_TZINT_ISR                
0     0013e9c4  _EPWM6_INT_ISR                  
0     0013e974  _EPWM6_TZINT_ISR                
0     0013e9ce  _EPWM7_INT_ISR                  
0     0013e97e  _EPWM7_TZINT_ISR                
0     0013e9d8  _EPWM8_INT_ISR                  
0     0013e988  _EPWM8_TZINT_ISR                
0     0013ea46  _EPWM9_INT_ISR                  
0     0013ea1e  _EPWM9_TZINT_ISR                
1     00005100  _EPwm1Regs                      
1     00005180  _EPwm2Regs                      
1     00005200  _EPwm3Regs                      
1     00005280  _EPwm4Regs                      
1     00005300  _EPwm5Regs                      
1     00005380  _EPwm6Regs                      
1     00005400  _EPwm7Regs                      
1     00005480  _EPwm8Regs                      
1     00005500  _EPwm9Regs                      
0     0013ea28  _EQEP1_INT_ISR                  
0     0013ea32  _EQEP2_INT_ISR                  
0     0013ea3c  _EQEP3_INT_ISR                  
1     00005b00  _EQep1Regs                      
1     00005b40  _EQep2Regs                      
1     00005b80  _EQep3Regs                      
1     0013fff4  _EcslPwl                        
0     0013f0c6  _EcslUnlock                     
0     0013f52a  _EnableInterrupts               
1     00004430  _EpiRegs                        
0     0013f3e6  _Error                          
1     0000a580  _ErrorCount                     
1     0000a4c1  _ErrorFlag                      
1     0000a3aa  _FAULT_WARNING                  
1     00004000  _FlashCtrlRegs                  
1     00004300  _FlashEccRegs                   
1     0013fff2  _FlashExeOnly                   
0     0000804e  _FlashGainPump                  
0     0000805b  _FlashLeavePump                 
0     0013e195  _GPIOConfig                     
0     0013ec2a  _GPIO_InputTest                 
0     0013ed6d  _GPIO_OutputTest                
0     0013f0e5  _GetEXEstatus                   
1     00005f80  _GpioCtrlRegs                   
1     00005fc0  _GpioDataRegs                   
1     00005f80  _GpioG1CtrlRegs                 
1     00005fc0  _GpioG1DataRegs                 
1     00005fe0  _GpioG1TripRegs                 
1     00006f80  _GpioG2CtrlRegs                 
1     00006fc0  _GpioG2DataRegs                 
1     00005fe0  _GpioTripRegs                   
0     0013eab4  _I2CINT1A_ISR                   
0     0013eabe  _I2CINT2A_ISR                   
1     00007900  _I2caRegs                       
0     0013e884  _ILLEGAL_ISR                    
0     0013e848  _INT13_ISR                      
0     0013e852  _INT14_ISR                      
0     0013e48c  _IPCCInitialize                 
0     0013e61a  _IPCCtoMBlockRead               
0     0013e63a  _IPCCtoMBlockWrite              
0     0013e654  _IPCCtoMBlockWrite_Protected    
0     0013e5c0  _IPCCtoMClearBits               
0     0013e5d6  _IPCCtoMClearBits_Protected     
0     0013e558  _IPCCtoMDataRead                
0     0013e576  _IPCCtoMDataRead_Protected      
0     0013e5ec  _IPCCtoMDataWrite               
0     0013e603  _IPCCtoMDataWrite_Protected     
0     0013f2dd  _IPCCtoMFlagBusy                
0     0013f2f4  _IPCCtoMFlagClear               
0     0013f2ec  _IPCCtoMFlagSet                 
0     0013e66e  _IPCCtoMFunctionCall            
0     0013e697  _IPCCtoMReqMemAccess            
0     0013e682  _IPCCtoMSendMessage             
0     0013e594  _IPCCtoMSetBits                 
0     0013e5aa  _IPCCtoMSetBits_Protected       
0     0013f2fc  _IPCCtoMSharedRamConvert        
1     0000a4c0  _IPCDataReceiveFlag             
0     0013e7a6  _IPCMtoCBlockRead               
0     0013e7c8  _IPCMtoCBlockWrite              
0     0013e802  _IPCMtoCBlockWrite_Protected    
0     0013e777  _IPCMtoCClearBits               
0     0013e78d  _IPCMtoCClearBits_Protected     
0     0013e708  _IPCMtoCDataRead                
0     0013e72a  _IPCMtoCDataRead_Protected      
0     0013e6cd  _IPCMtoCDataWrite               
0     0013e6e9  _IPCMtoCDataWrite_Protected     
0     0013f2c6  _IPCMtoCFlagAcknowledge         
0     0013f2ce  _IPCMtoCFlagBusy                
0     0013e83f  _IPCMtoCFunctionCall            
0     0013e74c  _IPCMtoCSetBits                 
0     0013e760  _IPCMtoCSetBits_Protected       
1     0000a500  _IPCRecievedBuffer              
0     0013f388  _IPC_FlagStatus                 
0     0013f35f  _IPC_Initialize                 
0     0013f3c2  _IPC_Read                       
0     0013f393  _IPC_Write                      
0     0013f3f2  _InitCpuTimers                  
0     0013e2b7  _InitDebugLED                   
0     0013e2cf  _InitEPwm1                      
0     0013e329  _InitEPwm2                      
0     0013e37d  _InitEPwm4                      
0     0013e3d6  _InitEPwm5                      
0     00008000  _InitFlash                      
0     0013f55c  _InitGpio                       
0     0013e223  _InitIPC                        
0     0013e42d  _InitNMI                        
0     0013f04a  _InitPeripheralClocks           
0     0013f506  _InitPieCtrl                    
0     0013f5a4  _InitPieVectTable               
0     0013e27c  _InitSCI                        
0     0013eff6  _InitSysCtrl                    
0     0013e000  _InitSystem                     
0     0013e23b  _InitTimer                      
0     0013e519  _IpcGet                         
0     0013e4e1  _IpcPut                         
0     0013f326  _IpcSync                        
0     0013eb7c  _LUF_ISR                        
0     0013eb72  _LVF_ISR                        
0     0013f0dd  _LockDevice                     
1     0000a584  _LoopCount                      
1     00004400  _M3PllRegs                      
0     0013ea64  _MRINTA_ISR                     
1     0000a001  _MS_Delay                       
0     0013eb18  _MTOCIPC_INT1_ISR               
0     0013eb22  _MTOCIPC_INT2_ISR               
0     0013eb2c  _MTOCIPC_INT3_ISR               
0     0013eb36  _MTOCIPC_INT4_ISR               
0     0013ea6e  _MXINTA_ISR                     
1     00005000  _McbspaRegs                     
0     0013f110  _MtoCIPC1IntHandler             
0     0013f197  _MtoCIPC2IntHandler             
0     0013e87a  _NMI_ISR                        
1     00007060  _NmiIntruptRegs                 
0     0013eb93  _PIE_RESERVED                   
0     0013eba7  _ParseCommand                   
1     00000ce0  _PieCtrlRegs                    
1     00000d00  _PieVectTable                   
1     00000e00  _PieVectTableCopy               
0     0013fa92  _PieVectTableInit               
1     00004a00  _RAMErrRegs                     
1     00004900  _RAMRegs                        
0     0013e866  _RTOSINT_ISR                    
0     0013806a  _RamfuncsLoadEnd                
abs   0000006a  _RamfuncsLoadSize               
0     00138000  _RamfuncsLoadStart              
0     0000806a  _RamfuncsRunEnd                 
abs   0000006a  _RamfuncsRunSize                
0     00008000  _RamfuncsRunStart               
0     0013eac8  _SCIRXINTA_ISR                  
0     0013eef0  _SCIRxINTA_ISR                  
0     0013ead2  _SCITXINTA_ISR                  
0     0013ea50  _SPIRXINTA_ISR                  
0     0013ea5a  _SPITXINTA_ISR                  
1     00007050  _SciaRegs                       
0     0013f34f  _SendIpcCommand                 
0     0013f31e  _SendIpcFlag                    
0     00008025  _SetupFlash                     
1     00007040  _SpiaRegs                       
1     00007010  _SysCtrlRegs                    
0     0013e92e  _TINT0_ISR                      
0     0013e8e8  _USER10_ISR                     
0     0013e8f2  _USER11_ISR                     
0     0013e8fc  _USER12_ISR                     
0     0013e88e  _USER1_ISR                      
0     0013e898  _USER2_ISR                      
0     0013e8a2  _USER3_ISR                      
0     0013e8ac  _USER4_ISR                      
0     0013e8b6  _USER5_ISR                      
0     0013e8c0  _USER6_ISR                      
0     0013e8ca  _USER7_ISR                      
0     0013e8d4  _USER8_ISR                      
0     0013e8de  _USER9_ISR                      
0     0013ebee  _UnitTest                       
0     0013e938  _WAKEINT_ISR                    
0     0013f344  _WaitForIpcAck                  
0     0013f310  _WaitForIpcFlag                 
0     0013e91a  _XINT1_ISR                      
0     0013e924  _XINT2_ISR                      
0     0013eb40  _XINT3_ISR                      
1     00007070  _XIntruptRegs                   
1     00000700  __STACK_END                     
abs   00000300  __STACK_SIZE                    
1     0000a3a6  ___TI_cleanup_ptr               
1     0000a3a8  ___TI_dtors_ptr                 
1     0000a3a4  ___TI_enable_exit_profile_output
abs   ffffffff  ___TI_pprof_out_hndl            
abs   ffffffff  ___TI_prof_data_size            
abs   ffffffff  ___TI_prof_data_start           
abs   ffffffff  ___binit__                      
abs   ffffffff  ___c_args__                     
0     0013fc44  ___cinit__                      
0     0013f611  ___etext__                      
abs   ffffffff  ___pinit__                      
0     0013e000  ___text__                       
0     0013f5e2  __args_main                     
1     0000a3ac  __lock                          
0     0013f60d  __nop                           
0     0013f609  __register_lock                 
0     0013f605  __register_unlock               
1     00000400  __stack                         
0     0013f610  __system_post_cinit             
0     0013f60e  __system_pre_init               
1     0000a3ae  __unlock                        
1     0000a100  _aADC1ChannelTest               
1     0000a080  _aADC1Test                      
1     0000a058  _aADC1TestFail                  
1     0000a017  _aADC1TestSuccess               
1     0000a1c0  _aEndTestMsg                    
1     0000a040  _aFailGPIOInputTest             
1     0000a002  _aInitMsg                       
1     0000a180  _aRxBufferSCI                   
1     0000a0c0  _aStartGPIOInputTest            
1     0000a240  _aStartMsg                      
1     0000a140  _aStartTestMsg                  
1     0000a09a  _aSuccessGPIOInputTest          
0     0013f533  _abort                          
1     0000a454  _adc1Voltage_ChannelA0          
1     0000a440  _adc1Voltage_ChannelA2          
1     0000a480  _adc1Voltage_ChannelA3          
1     0000a468  _adc1Voltage_ChannelA4          
1     0000a3e0  _adc1Voltage_ChannelA6          
1     0000a3cc  _adc1Voltage_ChannelA7          
1     0000a3f4  _adc1Voltage_ChannelB0          
1     0000a41e  _adc1Voltage_ChannelB3          
1     0000a432  _adc1Voltage_ChannelB4          
1     0000a40a  _adc1Voltage_ChannelB7          
0     0013f1f4  _adc1_isr                       
1     0000a45e  _adc2Voltage_ChannelA0          
1     0000a44a  _adc2Voltage_ChannelA2          
1     0000a48a  _adc2Voltage_ChannelA3          
1     0000a3ea  _adc2Voltage_ChannelA4          
1     0000a428  _adc2Voltage_ChannelA6          
1     0000a3c2  _adc2Voltage_ChannelA7          
1     0000a3d6  _adc2Voltage_ChannelB0          
1     0000a400  _adc2Voltage_ChannelB3          
1     0000a414  _adc2Voltage_ChannelB4          
1     0000a472  _adc2Voltage_ChannelB7          
0     0013f24b  _adc2_isr                       
0     0013f46d  _c_int00                        
0     0013f580  _copy_in                        
1     0000a586  _count                          
1     0000a587  _counter                        
0     0013ee62  _cpu_timer0_isr                 
0     0013eec0  _cpu_timer1_isr                 
0     0013eedb  _cpu_timer2_isr                 
1     0000a588  _dataStore                      
1     0000a58a  _dataStore1                     
1     0000a000  _enModuleTest                   
0     0013ef3d  _epwm1_isr                      
0     0013ef52  _epwm2_isr                      
0     0013ef67  _epwm4_isr                      
0     0013ef7c  _epwm5_isr                      
0     0013f535  _exit                           
1     0003f800  _g_asIPCCtoMBuffers             
0     0003fc00  _g_asIPCMtoCBuffers             
1     0000a4c6  _g_sIpcController1              
1     0000a4d4  _g_sIpcController2              
1     0003f884  _g_usGetReadIndexes             
0     0003fc80  _g_usGetWriteIndexes            
0     0003fc84  _g_usPutReadIndexes             
1     0003f880  _g_usPutWriteIndexes            
0     0013f3e7  _getIPCDataRecieveStatus        
1     0000a585  _i                              
1     0000a58c  _ipcData                        
1     0000a583  _loop                           
0     0013f4c3  _main                           
0     0013f5c4  _memcpy                         
1     0000a4c2  _pulMsgRam                      
1     0000a4c4  _pulMsgRam_M3                   
1     0000a5c0  _rdata                          
0     0013eb9d  _rsvd_ISR                       
0     0013f4fe  _scia_fifo_init                 
0     0013f4eb  _scia_msg                       
0     0013f4de  _scia_xmit                      
0     0013f3eb  _setIPCDataRecieveStatus        
0     0013f5fb  _strcmp                         
1     0000a581  _tempVal                        
1     0000a582  _timerOut                       
0     0013ef91  _xint1_isr                      
0     0013efa2  _xint2_isr                      
0     0013efb7  _xint3_isr                      
abs   ffffffff  binit                           
0     0013fc44  cinit                           
0     0013fff0  code_start                      
0     0013f611  etext                           
abs   ffffffff  pinit                           


GLOBAL SYMBOLS: SORTED BY Symbol Address 

page  address   name                            
----  -------   ----                            
0     00008000  _InitFlash                      
0     00008000  _RamfuncsRunStart               
0     00008025  _SetupFlash                     
0     0000804e  _FlashGainPump                  
0     0000805b  _FlashLeavePump                 
0     00008066  _DSP28x_usDelay                 
0     0000806a  _RamfuncsRunEnd                 
0     0003fc00  _g_asIPCMtoCBuffers             
0     0003fc80  _g_usGetWriteIndexes            
0     0003fc84  _g_usPutReadIndexes             
0     00138000  _RamfuncsLoadStart              
0     0013806a  _RamfuncsLoadEnd                
0     0013e000  .text                           
0     0013e000  _InitSystem                     
0     0013e000  ___text__                       
0     0013e034  _Adc1Config                     
0     0013e0a8  _Adc2Config                     
0     0013e152  _AdcSocPWM                      
0     0013e195  _GPIOConfig                     
0     0013e223  _InitIPC                        
0     0013e23b  _InitTimer                      
0     0013e27c  _InitSCI                        
0     0013e2b7  _InitDebugLED                   
0     0013e2cf  _InitEPwm1                      
0     0013e329  _InitEPwm2                      
0     0013e37d  _InitEPwm4                      
0     0013e3d6  _InitEPwm5                      
0     0013e42d  _InitNMI                        
0     0013e48c  _IPCCInitialize                 
0     0013e4e1  _IpcPut                         
0     0013e519  _IpcGet                         
0     0013e558  _IPCCtoMDataRead                
0     0013e576  _IPCCtoMDataRead_Protected      
0     0013e594  _IPCCtoMSetBits                 
0     0013e5aa  _IPCCtoMSetBits_Protected       
0     0013e5c0  _IPCCtoMClearBits               
0     0013e5d6  _IPCCtoMClearBits_Protected     
0     0013e5ec  _IPCCtoMDataWrite               
0     0013e603  _IPCCtoMDataWrite_Protected     
0     0013e61a  _IPCCtoMBlockRead               
0     0013e63a  _IPCCtoMBlockWrite              
0     0013e654  _IPCCtoMBlockWrite_Protected    
0     0013e66e  _IPCCtoMFunctionCall            
0     0013e682  _IPCCtoMSendMessage             
0     0013e697  _IPCCtoMReqMemAccess            
0     0013e6cd  _IPCMtoCDataWrite               
0     0013e6e9  _IPCMtoCDataWrite_Protected     
0     0013e708  _IPCMtoCDataRead                
0     0013e72a  _IPCMtoCDataRead_Protected      
0     0013e74c  _IPCMtoCSetBits                 
0     0013e760  _IPCMtoCSetBits_Protected       
0     0013e777  _IPCMtoCClearBits               
0     0013e78d  _IPCMtoCClearBits_Protected     
0     0013e7a6  _IPCMtoCBlockRead               
0     0013e7c8  _IPCMtoCBlockWrite              
0     0013e802  _IPCMtoCBlockWrite_Protected    
0     0013e83f  _IPCMtoCFunctionCall            
0     0013e848  _INT13_ISR                      
0     0013e852  _INT14_ISR                      
0     0013e85c  _DATALOG_ISR                    
0     0013e866  _RTOSINT_ISR                    
0     0013e870  _EMUINT_ISR                     
0     0013e87a  _NMI_ISR                        
0     0013e884  _ILLEGAL_ISR                    
0     0013e88e  _USER1_ISR                      
0     0013e898  _USER2_ISR                      
0     0013e8a2  _USER3_ISR                      
0     0013e8ac  _USER4_ISR                      
0     0013e8b6  _USER5_ISR                      
0     0013e8c0  _USER6_ISR                      
0     0013e8ca  _USER7_ISR                      
0     0013e8d4  _USER8_ISR                      
0     0013e8de  _USER9_ISR                      
0     0013e8e8  _USER10_ISR                     
0     0013e8f2  _USER11_ISR                     
0     0013e8fc  _USER12_ISR                     
0     0013e906  _ADCINT1_ISR                    
0     0013e910  _ADCINT2_ISR                    
0     0013e91a  _XINT1_ISR                      
0     0013e924  _XINT2_ISR                      
0     0013e92e  _TINT0_ISR                      
0     0013e938  _WAKEINT_ISR                    
0     0013e942  _EPWM1_TZINT_ISR                
0     0013e94c  _EPWM2_TZINT_ISR                
0     0013e956  _EPWM3_TZINT_ISR                
0     0013e960  _EPWM4_TZINT_ISR                
0     0013e96a  _EPWM5_TZINT_ISR                
0     0013e974  _EPWM6_TZINT_ISR                
0     0013e97e  _EPWM7_TZINT_ISR                
0     0013e988  _EPWM8_TZINT_ISR                
0     0013e992  _EPWM1_INT_ISR                  
0     0013e99c  _EPWM2_INT_ISR                  
0     0013e9a6  _EPWM3_INT_ISR                  
0     0013e9b0  _EPWM4_INT_ISR                  
0     0013e9ba  _EPWM5_INT_ISR                  
0     0013e9c4  _EPWM6_INT_ISR                  
0     0013e9ce  _EPWM7_INT_ISR                  
0     0013e9d8  _EPWM8_INT_ISR                  
0     0013e9e2  _ECAP1_INT_ISR                  
0     0013e9ec  _ECAP2_INT_ISR                  
0     0013e9f6  _ECAP3_INT_ISR                  
0     0013ea00  _ECAP4_INT_ISR                  
0     0013ea0a  _ECAP5_INT_ISR                  
0     0013ea14  _ECAP6_INT_ISR                  
0     0013ea1e  _EPWM9_TZINT_ISR                
0     0013ea28  _EQEP1_INT_ISR                  
0     0013ea32  _EQEP2_INT_ISR                  
0     0013ea3c  _EQEP3_INT_ISR                  
0     0013ea46  _EPWM9_INT_ISR                  
0     0013ea50  _SPIRXINTA_ISR                  
0     0013ea5a  _SPITXINTA_ISR                  
0     0013ea64  _MRINTA_ISR                     
0     0013ea6e  _MXINTA_ISR                     
0     0013ea78  _DINTCH1_ISR                    
0     0013ea82  _DINTCH2_ISR                    
0     0013ea8c  _DINTCH3_ISR                    
0     0013ea96  _DINTCH4_ISR                    
0     0013eaa0  _DINTCH5_ISR                    
0     0013eaaa  _DINTCH6_ISR                    
0     0013eab4  _I2CINT1A_ISR                   
0     0013eabe  _I2CINT2A_ISR                   
0     0013eac8  _SCIRXINTA_ISR                  
0     0013ead2  _SCITXINTA_ISR                  
0     0013eadc  _ADCINT3_ISR                    
0     0013eae6  _ADCINT4_ISR                    
0     0013eaf0  _ADCINT5_ISR                    
0     0013eafa  _ADCINT6_ISR                    
0     0013eb04  _ADCINT7_ISR                    
0     0013eb0e  _ADCINT8_ISR                    
0     0013eb18  _MTOCIPC_INT1_ISR               
0     0013eb22  _MTOCIPC_INT2_ISR               
0     0013eb2c  _MTOCIPC_INT3_ISR               
0     0013eb36  _MTOCIPC_INT4_ISR               
0     0013eb40  _XINT3_ISR                      
0     0013eb4a  _CFLSINGERR_ISR                 
0     0013eb54  _CFLFSM_ISR                     
0     0013eb5e  _CRAMSINGERR_ISR                
0     0013eb68  _CRAMACCVIOL_ISR                
0     0013eb72  _LVF_ISR                        
0     0013eb7c  _LUF_ISR                        
0     0013eb86  _EMPTY_ISR                      
0     0013eb93  _PIE_RESERVED                   
0     0013eb9d  _rsvd_ISR                       
0     0013eba7  _ParseCommand                   
0     0013ebee  _UnitTest                       
0     0013ec15  _ADC_Test                       
0     0013ec2a  _GPIO_InputTest                 
0     0013ed6d  _GPIO_OutputTest                
0     0013ee62  _cpu_timer0_isr                 
0     0013eec0  _cpu_timer1_isr                 
0     0013eedb  _cpu_timer2_isr                 
0     0013eef0  _SCIRxINTA_ISR                  
0     0013ef3d  _epwm1_isr                      
0     0013ef52  _epwm2_isr                      
0     0013ef67  _epwm4_isr                      
0     0013ef7c  _epwm5_isr                      
0     0013ef91  _xint1_isr                      
0     0013efa2  _xint2_isr                      
0     0013efb7  _xint3_isr                      
0     0013eff6  _InitSysCtrl                    
0     0013f04a  _InitPeripheralClocks           
0     0013f0a5  _CsmUnlock                      
0     0013f0c6  _EcslUnlock                     
0     0013f0dd  _LockDevice                     
0     0013f0e5  _GetEXEstatus                   
0     0013f0f8  _CSMSecurityStatus              
0     0013f104  _ECSLSecurityStatus             
0     0013f110  _MtoCIPC1IntHandler             
0     0013f197  _MtoCIPC2IntHandler             
0     0013f1f4  _adc1_isr                       
0     0013f24b  _adc2_isr                       
0     0013f2c6  _IPCMtoCFlagAcknowledge         
0     0013f2ce  _IPCMtoCFlagBusy                
0     0013f2dd  _IPCCtoMFlagBusy                
0     0013f2ec  _IPCCtoMFlagSet                 
0     0013f2f4  _IPCCtoMFlagClear               
0     0013f2fc  _IPCCtoMSharedRamConvert        
0     0013f310  _WaitForIpcFlag                 
0     0013f31e  _SendIpcFlag                    
0     0013f326  _IpcSync                        
0     0013f33c  _AckIpcFlag                     
0     0013f344  _WaitForIpcAck                  
0     0013f34f  _SendIpcCommand                 
0     0013f35f  _IPC_Initialize                 
0     0013f388  _IPC_FlagStatus                 
0     0013f393  _IPC_Write                      
0     0013f3c2  _IPC_Read                       
0     0013f3e6  _Error                          
0     0013f3e7  _getIPCDataRecieveStatus        
0     0013f3eb  _setIPCDataRecieveStatus        
0     0013f3f2  _InitCpuTimers                  
0     0013f433  _ConfigCpuTimer                 
0     0013f46d  _c_int00                        
0     0013f4c3  _main                           
0     0013f4de  _scia_xmit                      
0     0013f4eb  _scia_msg                       
0     0013f4fe  _scia_fifo_init                 
0     0013f506  _InitPieCtrl                    
0     0013f52a  _EnableInterrupts               
0     0013f533  C$$EXIT                         
0     0013f533  _abort                          
0     0013f535  _exit                           
0     0013f55c  _InitGpio                       
0     0013f580  _copy_in                        
0     0013f5a4  _InitPieVectTable               
0     0013f5c4  _memcpy                         
0     0013f5e2  __args_main                     
0     0013f5fb  _strcmp                         
0     0013f605  __register_unlock               
0     0013f609  __register_lock                 
0     0013f60d  __nop                           
0     0013f60e  __system_pre_init               
0     0013f610  __system_post_cinit             
0     0013f611  ___etext__                      
0     0013f611  etext                           
0     0013fa92  _PieVectTableInit               
0     0013fc44  ___cinit__                      
0     0013fc44  cinit                           
0     0013fff0  code_start                      
1     00000400  __stack                         
1     00000700  __STACK_END                     
1     00000880  _DevEmuRegs                     
1     00000ae0  _CsmRegs                        
1     00000b00  _Adc1Result                     
1     00000b00  _AdcResult                      
1     00000b40  _Adc2Result                     
1     00000c00  _CpuTimer0Regs                  
1     00000c08  _CpuTimer1Regs                  
1     00000c10  _CpuTimer2Regs                  
1     00000ce0  _PieCtrlRegs                    
1     00000d00  _PieVectTable                   
1     00000e00  _PieVectTableCopy               
1     00001000  _DmaRegs                        
1     00001700  _AnalogSysctrlRegs              
1     00004000  _FlashCtrlRegs                  
1     00004300  _FlashEccRegs                   
1     00004400  _M3PllRegs                      
1     00004430  _EpiRegs                        
1     00004900  _RAMRegs                        
1     00004a00  _RAMErrRegs                     
1     00004e00  _CtoMIpcRegs                    
1     00005000  _McbspaRegs                     
1     00005100  _EPwm1Regs                      
1     00005180  _EPwm2Regs                      
1     00005200  _EPwm3Regs                      
1     00005280  _EPwm4Regs                      
1     00005300  _EPwm5Regs                      
1     00005380  _EPwm6Regs                      
1     00005400  _EPwm7Regs                      
1     00005480  _EPwm8Regs                      
1     00005500  _EPwm9Regs                      
1     00005a00  _ECap1Regs                      
1     00005a20  _ECap2Regs                      
1     00005a40  _ECap3Regs                      
1     00005a60  _ECap4Regs                      
1     00005a80  _ECap5Regs                      
1     00005aa0  _ECap6Regs                      
1     00005b00  _EQep1Regs                      
1     00005b40  _EQep2Regs                      
1     00005b80  _EQep3Regs                      
1     00005f80  _GpioCtrlRegs                   
1     00005f80  _GpioG1CtrlRegs                 
1     00005fc0  _GpioDataRegs                   
1     00005fc0  _GpioG1DataRegs                 
1     00005fe0  _GpioG1TripRegs                 
1     00005fe0  _GpioTripRegs                   
1     00006400  _Comp1Regs                      
1     00006420  _Comp2Regs                      
1     00006440  _Comp3Regs                      
1     00006460  _Comp4Regs                      
1     00006480  _Comp5Regs                      
1     000064a0  _Comp6Regs                      
1     00006f80  _GpioG2CtrlRegs                 
1     00006fc0  _GpioG2DataRegs                 
1     00007010  _SysCtrlRegs                    
1     00007040  _SpiaRegs                       
1     00007050  _SciaRegs                       
1     00007060  _NmiIntruptRegs                 
1     00007070  _XIntruptRegs                   
1     00007100  _Adc1Regs                       
1     00007100  _AdcRegs                        
1     00007180  _Adc2Regs                       
1     00007900  _I2caRegs                       
1     0000a000  _enModuleTest                   
1     0000a001  _MS_Delay                       
1     0000a002  _aInitMsg                       
1     0000a017  _aADC1TestSuccess               
1     0000a040  _aFailGPIOInputTest             
1     0000a058  _aADC1TestFail                  
1     0000a080  _aADC1Test                      
1     0000a09a  _aSuccessGPIOInputTest          
1     0000a0c0  _aStartGPIOInputTest            
1     0000a100  _aADC1ChannelTest               
1     0000a140  _aStartTestMsg                  
1     0000a180  _aRxBufferSCI                   
1     0000a1c0  _aEndTestMsg                    
1     0000a240  _aStartMsg                      
1     0000a38c  _CpuTimer1                      
1     0000a394  _CpuTimer2                      
1     0000a39c  _CpuTimer0                      
1     0000a3a4  ___TI_enable_exit_profile_output
1     0000a3a6  ___TI_cleanup_ptr               
1     0000a3a8  ___TI_dtors_ptr                 
1     0000a3aa  _FAULT_WARNING                  
1     0000a3ac  __lock                          
1     0000a3ae  __unlock                        
1     0000a3c0  _ConversionCount                
1     0000a3c1  _ConversionCount1               
1     0000a3c2  _adc2Voltage_ChannelA7          
1     0000a3cc  _adc1Voltage_ChannelA7          
1     0000a3d6  _adc2Voltage_ChannelB0          
1     0000a3e0  _adc1Voltage_ChannelA6          
1     0000a3ea  _adc2Voltage_ChannelA4          
1     0000a3f4  _adc1Voltage_ChannelB0          
1     0000a400  _adc2Voltage_ChannelB3          
1     0000a40a  _adc1Voltage_ChannelB7          
1     0000a414  _adc2Voltage_ChannelB4          
1     0000a41e  _adc1Voltage_ChannelB3          
1     0000a428  _adc2Voltage_ChannelA6          
1     0000a432  _adc1Voltage_ChannelB4          
1     0000a440  _adc1Voltage_ChannelA2          
1     0000a44a  _adc2Voltage_ChannelA2          
1     0000a454  _adc1Voltage_ChannelA0          
1     0000a45e  _adc2Voltage_ChannelA0          
1     0000a468  _adc1Voltage_ChannelA4          
1     0000a472  _adc2Voltage_ChannelB7          
1     0000a480  _adc1Voltage_ChannelA3          
1     0000a48a  _adc2Voltage_ChannelA3          
1     0000a4c0  _IPCDataReceiveFlag             
1     0000a4c1  _ErrorFlag                      
1     0000a4c2  _pulMsgRam                      
1     0000a4c4  _pulMsgRam_M3                   
1     0000a4c6  _g_sIpcController1              
1     0000a4d4  _g_sIpcController2              
1     0000a500  _IPCRecievedBuffer              
1     0000a580  _ErrorCount                     
1     0000a581  _tempVal                        
1     0000a582  _timerOut                       
1     0000a583  _loop                           
1     0000a584  _LoopCount                      
1     0000a585  _i                              
1     0000a586  _count                          
1     0000a587  _counter                        
1     0000a588  _dataStore                      
1     0000a58a  _dataStore1                     
1     0000a58c  _ipcData                        
1     0000a5c0  _rdata                          
1     0003f800  _g_asIPCCtoMBuffers             
1     0003f880  _g_usPutWriteIndexes            
1     0003f884  _g_usGetReadIndexes             
1     0013fff2  _FlashExeOnly                   
1     0013fff4  _EcslPwl                        
1     0013fff8  _CsmPwl                         
abs   0000006a  _RamfuncsLoadSize               
abs   0000006a  _RamfuncsRunSize                
abs   00000300  __STACK_SIZE                    
abs   ffffffff  ___TI_pprof_out_hndl            
abs   ffffffff  ___TI_prof_data_size            
abs   ffffffff  ___TI_prof_data_start           
abs   ffffffff  ___binit__                      
abs   ffffffff  ___c_args__                     
abs   ffffffff  ___pinit__                      
abs   ffffffff  binit                           
abs   ffffffff  pinit                           

[364 symbols]
